S023000064656D6F70726F675F6E75636C656F5F73746D33326631303372622E73726563D9
S3150800200000500020A1310008F1310008F131000824
S31508002010F1310008F1310008F13100080000000034
S31508002020000000000000000000000000F131000878
S31508002030F131000800000000F131000829320008DB
S31508002040F1310008F1310008F1310008F1310008DA
S31508002050F1310008F1310008F1310008F1310008CA
S31508002060F1310008F1310008F1310008F1310008BA
S31508002070F1310008F1310008F1310008F1310008AA
S31508002080F1310008F1310008F1310008F13100089A
S31508002090F1310008F1310008F1310008F13100088A
S315080020A0F1310008F1310008F1310008F13100087A
S315080020B0F1310008F1310008F1310008F13100086A
S315080020C0F1310008F1310008F1310008F13100085A
S315080020D0F1310008F1310008F1310008F13100084A
S315080020E0F1310008F1310008F13100080000000064
S315080020F000000000000000000000000000000000D2
S3150800210000000000000000005FF808F1EE11AA5573
S3150800211010B5054C237833B9044B13B10448AFF313
S3150800212000800123237010BD0C0000200000000071
S315080021307C32000808B5034B1BB103490348AFF3CB
S31508002140008008BD00000000100000207C32000856
S3150800215008B50848084B03604FF461434360002301
S315080021608360C360036183610C224261C36100F02E
S3150800217088FE08BD280000200044004008B500235A
S3150800218001220146034800F0ABFE08B1002008BD55
S31508002190012008BD2800002008B5FFF7D9FF08BDB3
S315080021A0BFF34F8F0549CA6802F4E062044B134334
S315080021B0CB60BFF34F8F00BFFDE700BF00ED00E027
S315080021C00400FA0508B5214B1B78B3B92048FFF778
S315080021D0D5FF012800D008BD1D4B1B78013BDBB29B
S315080021E03F2BF8D801F01CF81A4B18600122174B40
S315080021F01A700022184B1A7008BD174B1B7801334A
S3150800220013481844FFF7BAFF01280AD001F008F866
S31508002210104B1B6864339842DDD900220B4B1A70A9
S31508002220D9E70D4A13780133DBB21370084A1278DE
S315080022309342D0D10021054A1170054A5278FF2AE7
S31508002240C9D1022BC7D1FFF7ABFF00BFA9000020F9
S3150800225068000020AC000020AA00002008B5FFF79F
S31508002260B1FF08BD08B500222021024800F0DAF9BE
S3150800227008BD00BF0008014010B500F0D1FF0E4BA5
S315080022801B68C31AB3F5FA7F0CD304460B4B1B78AD
S315080022904BB90122094B1A702021094800F0C2F9EE
S315080022A0054B1C6010BD0022044B1A7020210448FF
S315080022B000F0B8F9F4E700BFB4000020B000002031
S315080022C00008014010B504460E4B18784FF47A738F
S315080022D0B3FBF0F30C4A1068B0FBF3F000F080F89B
S315080022E068B90F2C01D9012010BD002221464FF0F4
S315080022F0FF3000F043F8054B1C60002010BD01209C
S3150800230010BD00BF000000200800002004000020C7
S3150800231008B5074A136843F010031360032000F05A
S315080023201BF80020FFF7CEFF00F0BCFE002008BD1A
S3150800233000200240034A1168034B1B780B441360C4
S31508002340704700BFB800002000000020014B186845
S31508002350704700BFB8000020074AD36823F4E0633B
S315080023601B041B0C000200F4E060184340F0BF6039
S3150800237040F40030D060704700ED00E030B4164BF2
S31508002380DB68C3F30223C3F10704042C28BF042423
S315080023901D1D062D17D9033B012505FA04F4013C3A
S315080023A02140994005FA03F3013B134019430028DD
S315080023B00BDB0901C9B200F1604000F5614080F805
S315080023C0001330BC70470023E6E700F00F00090150
S315080023D0C9B2024B1954F4E700ED00E014ED00E031
S315080023E00138B0F1807F0AD2064B5860F021064AC0
S315080023F082F823100020986007221A60704701208F
S31508002400704700BF10E000E000ED00E0042805D0AA
S31508002410054A136823F0040313607047024A1368D9
S3150800242043F004031360704710E000E0704708B5F6
S31508002430FFF7FCFF08BD0000F0B583B00026344660
S3150800244071E0002D00F0A180012D00D1CE68FF2B90
S3150800245000F2AF808646FF2B00F2AE80A500DEF8BC
S3150800246000200F27AF4022EA070206FA05F52A439D
S31508002470CEF800204A6812F0805F53D0634A956907
S3150800248045F001059561926902F001020192019AEF
S31508002490A508AF1C5E4A52F8272004F00307BF00C0
S315080024A04FF00F0E0EFA07FE22EA0E02DFF870E171
S315080024B0704500F088800EF5806E704500F08680C5
S315080024C00EF5806E704500F084800EF5806E7045BE
S315080024D076D04FF0040E0EFA07F73A4302354C4F02
S315080024E047F825204A6812F4803F75D0494D2A6876
S315080024F01A432A604A6812F4003F73D0454D6A6849
S315080025001A436A604A6812F4801F71D0414DAA685E
S315080025101A43AA604A6812F4001F6FD03D4DEA6854
S315080025201343EB6001340F2C6ED80122A2400B68CE
S3150800253013409A42F6D14D68122D30D00BD8022D91
S315080025402AD07FF67EAF032D2FD0112D7FF47FAFD3
S31508002550CE6804367BE7304FBD4216D00CD92F4FD4
S31508002560BD4212D007F58037BD420ED0A7F58017B9
S31508002570BD427FF46CAF08E0A7F58017BD4204D0D2
S3150800258007F58037BD427FF462AF8D687DB1012DB6
S3150800259008D0426108265AE7CE68083657E7CE685B
S315080025A00C3654E70261082651E700264FE7042651
S315080025B04DE700F1040E4EE7A4F10805AD004EE71D
S315080025C04FF0030E87E74FF0000E84E74FF0010E39
S315080025D081E74FF0020E7EE70E4D2A6822EA0302D3
S315080025E02A6087E70B4D6A6822EA03026A6089E770
S315080025F0084DAA6822EA0302AA608BE7054DEA6835
S3150800260022EA0303EB608DE703B0F0BD0010024039
S3150800261000000140000401400000211000003110B4
S315080026200008014012B90904016170470161704749
S3150800263082B0084B1B68084AA2FB03235B0A00FB0F
S3150800264003F0019000BF019B5A1E0192002BF9D19D
S3150800265002B0704708000020D34D621070B582B0F2
S315080026600446036813F0010F3DD0AC4B5B6803F0DA
S315080026700C03042B2ED0A94B5B6803F00C03082B24
S3150800268023D06368B3F5803F51D0002B55D103F1B1
S31508002690804303F504331A6822F480321A601A68F4
S315080026A022F480221A606368002B60D0FFF74EFE82
S315080026B005469A4B1B6813F4003F14D1FFF746FEF4
S315080026C0401B6428F5D90320AFE1944B5B6813F4EB
S315080026D0803FD6D0914B1B6813F4003F03D0636844
S315080026E0002B00F09F81236813F0020F65D08B4BF7
S315080026F05B6813F00C0F4ED0884B5B6803F00C0335
S31508002700082B43D02369002B79D00122844B1A6009
S31508002710FFF71CFE0546814B1B6813F0020F65D1B7
S31508002720FFF714FE401B0228F5D903207DE17B4AFA
S31508002730136843F480331360B5E7B3F5A02F09D0C7
S31508002740764B1A6822F480321A601A6822F48022BC
S315080027501A60A8E703F18043A3F53C331A6842F4EC
S3150800276080221A601A6842F480321A609BE7FFF7E3
S31508002770EDFD0546694B1B6813F4003FB3D0FFF720
S31508002780E5FD401B6428F5D903204EE1634B5B68E1
S3150800279013F4803FB6D1614B1B6813F0020F04D0C7
S315080027A02369012B01D001203FE15C4A136823F01D
S315080027B0F803616943EAC1031360236813F0080F3D
S315080027C032D0A369002B6ED00122564B1A60FFF750
S315080027D0BDFD0546514B5B6A13F0020F21D1FFF789
S315080027E0B5FD401B0228F5D903201EE14B4A1368A4
S315080027F023F0F803616943EAC1031360DDE70022A9
S31508002800474B1A60FFF7A2FD0546444B1B6813F0B9
S31508002810020FD2D0FFF79AFD401B0228F5D90320F4
S3150800282003E10120FFF704FF236813F0040F00F00B
S3150800283099803A4BDB6913F0805F46D1374BDA69EA
S3150800284042F08052DA61DB6903F080530193019B01
S315080028500125354B1B6813F4807F38D0E368012BBC
S3150800286049D0002B4DD103F1804303F504331A6A8E
S3150800287022F001021A621A6A22F004021A62E36856
S31508002880002B5DD0FFF762FD0646244B1B6A13F04A
S31508002890020F66D1FFF75AFD801B41F28833984232
S315080028A0F3D90320C1E000221E4B1A60FFF74EFD44
S315080028B005461A4B5B6A13F0020FB5D0FFF746FDC3
S315080028C0401B0228F5D90320AFE00025C1E7164AC8
S315080028D0136843F480731360FFF738FD0646124BFE
S315080028E01B6813F4807FB9D1FFF730FD801B64287D
S315080028F0F5D9032099E0094A136A43F001031362E4
S31508002900BDE7052B12D0054B1A6A22F001021A629E
S315080029101A6A22F004021A62B1E700BF00100240E8
S31508002920000042428004424200700040414B1A6A4D
S3150800293042F004021A621A6A42F001021A629EE71B
S31508002940FFF704FD06463B4B1B6A13F0020F08D03F
S31508002950FFF7FCFC801B41F288339842F3D9032029
S3150800296063E0E5B9E369002B5ED0324A526802F0AB
S315080029700C02082A5BD0022B17D000222E4B1A60B5
S31508002980FFF7E4FC04462B4B1B6813F0007F47D087
S31508002990FFF7DCFC001B0228F5D9032045E0254A91
S315080029A0D36923F08053D361DCE70022224B1A60F7
S315080029B0FFF7CCFC05461F4B1B6813F0007F06D0BB
S315080029C0FFF7C4FC401B0228F5D903202DE0236A33
S315080029D0B3F5803F1AD017494B6823F47413226A5B
S315080029E0606A024313434B600122134B1A60FFF7D8
S315080029F0ADFC04460F4B1B6813F0007F0ED1FFF7A2
S31508002A00A5FC001B0228F5D903200EE0094A5368E5
S31508002A1023F40033A1680B435360DCE7002004E08D
S31508002A20002002E0012000E0002002B070BD012075
S31508002A30FBE700BF001002406000424210B586B0B6
S31508002A40154C94E80F000DF1180E0EE90F00238AB5
S31508002A50ADF80430114B5B6803F00C02082A18D154
S31508002A60C3F38342724412F8102C13F4803F03D147
S31508002A700B4800FB02F00DE0084B5B68C3F34043CC
S31508002A80734413F8143C074800FB02F0B0FBF3F05C
S31508002A9000E0044806B010BD943200080010024059
S31508002AA000093D0000127A00594B1B6803F0070322
S31508002AB08B420CD2564A136823F007030B43136064
S31508002AC0136803F00703994201D00120704770B5D7
S31508002AD0036813F0020F06D04E4A536823F0F0033A
S31508002AE08468234353600D460446036813F0010FB8
S31508002AF052D04368012B23D0022B28D0454A1268AE
S31508002B0012F0020F00F0828042494A6822F003025E
S31508002B1013434B60FFF71AFC06466368012B1DD06A
S31508002B20022B2AD03B4B5B6813F00C0F34D0FFF70F
S31508002B300DFC801B41F288339842F3D9032070BDFF
S31508002B40344A126812F4003FDED1012070BD314AC2
S31508002B50126812F0007FD7D1012070BD2D4B5B683B
S31508002B6003F00C03042B17D0FFF7F0FB801B41F290
S31508002B7088339842F2D9032070BD264B5B6803F070
S31508002B800C03082B08D0FFF7E1FB801B41F28833C2
S31508002B909842F2D9032070BD1D4B1B6803F007034A
S31508002BA09D420CD21A4A136823F007032B4313607D
S31508002BB0136803F007039D4201D0012070BD236806
S31508002BC013F0040F06D0134A536823F4E063E16850
S31508002BD00B435360236813F0080F07D00D4A536858
S31508002BE023F46053216943EAC1035360FFF726FFC4
S31508002BF0084B5B68C3F30313074AD35CD840074BFB
S31508002C0018600020FFF75EFB002070BD012070BD34
S31508002C100020024000100240A832000808000020E8
S31508002C20014B1868704700BF0800002008B5FFF779
S31508002C30F7FF044B5B68C3F30223034AD35CD8400F
S31508002C4008BD00BF00100240B832000808B5FFF7FB
S31508002C50E7FF044B5B68C3F3C223034AD35CD8403F
S31508002C6008BD00BF00100240B83200082DE9F04741
S31508002C7005460268136923F44053C1680B43136180
S31508002C80836802691343426913430168CA6822F4D8
S31508002C90B05222F00C021343CB600268536923F446
S31508002CA0407381690B435361D0F80080594B9845AE
S31508002CB057D0FFF7BBFF00EB800000EB80006C6885
S31508002CC0A400B0FBF4F4544FA7FB043464092601AE
S31508002CD0FFF7ACFF00EB800000EB80006C68A400F7
S31508002CE0B0FBF4FAFFF7A2FF00EB800000EB8000D0
S31508002CF06C68A400B0FBF4F4A7FB043464094FF035
S31508002D00640909FB14A424013234A7FB04346409BA
S31508002D1004F0F0043444FFF789FF00EB800000EB71
S31508002D2080006E68B600B0FBF6F6FFF77FFF00EB93
S31508002D30800000EB80006B689B00B0FBF3F0A7FBFC
S31508002D400030400909FB10694FEA091909F13209EF
S31508002D50A7FB0937C7F343172744C8F80870BDE827
S31508002D60F087FFF773FF00EB800000EB80006C68CC
S31508002D70A400B0FBF4F4284FA7FB04346409260129
S31508002D80FFF764FF00EB800000EB80006C68A4008E
S31508002D90B0FBF4FAFFF75AFF00EB800000EB800067
S31508002DA06C68A400B0FBF4F4A7FB043464094FF084
S31508002DB0640909FB14A424013234A7FB043464090A
S31508002DC004F0F0043444FFF741FF00EB800000EB09
S31508002DD080006E68B600B0FBF6F6FFF737FF00EB2B
S31508002DE0800000EB80006B689B00B0FBF3F3A7FB49
S31508002DF003235B0909FB13694FEA091909F132092B
S31508002E00A7FB0937C7F343172744C8F80870BDE876
S31508002E10F08700BF003801401F85EB512DE9F041CE
S31508002E2005460F4616469846069C2B681B6837EAE1
S31508002E3003030CBF01230023B3421ED1B4F1FF3FA5
S31508002E40F3D02CB1FFF782FAA0EB08008442ECD24B
S31508002E502A68D36823F4D073D3602A68536923F0A9
S31508002E6001035361202385F8393085F83A30002369
S31508002E7085F838300320BDE8F0810020BDE8F081F0
S31508002E80704758B310B5044690F839300BB324236D
S31508002E9084F839302268D36823F40053D360204677
S31508002EA0FFF7E4FE2268136923F49043136122684E
S31508002EB0536923F02A0353612268D36843F4005305
S31508002EC0D3600020E063202384F8393084F83A3050
S31508002ED010BD80F83830FFF7D3FFD8E701207047D8
S31508002EE02DE9F04182B01E4690F83A30DBB2202B2D
S31508002EF003D0022002B0BDE8F08104460D46904694
S31508002F00002958D0002A58D090F83830012B01D122
S31508002F100220EFE7012380F838300023C363222319
S31508002F2080F83A30FFF712FA0746A4F82C80A4F87E
S31508002F302E801DE000963B46002220212046FFF702
S31508002F406DFF00283BD1236933B923685B68C3F357
S31508002F50080325F8023B0BE023685B68DBB225F81B
S31508002F60013B05E023685B6803F07F032B7001359E
S31508002F70E38D9BB2C3B1E38D9BB2013B9BB2E38564
S31508002F80A368B3F5805FD5D000963B460022202182
S31508002F902046FFF743FFA0B92369002BE2D1236837
S31508002FA05B682B700135E3E7202384F83A3000206C
S31508002FB084F838009EE701209CE701209AE7032061
S31508002FC098E7032096E700000F4B1A6842F00102C3
S31508002FD01A6059680D4A0A405A601A6822F08472C3
S31508002FE022F480321A601A6822F480221A605A681B
S31508002FF022F4FE025A604FF41F029A604FF00062F4
S31508003000034B9A60704700BF001002400000FFF8AB
S3150800301000ED00E0014B024A9A60704700ED00E0BF
S315080030200020000800B591B0012306934FF4A022B2
S315080030300792002208920A9302230D934FF48033D5
S315080030400E934FF4E0130F9306A8FFF707FB00B1A2
S31508003050FEE70F23019302210291002303934FF405
S3150800306080620492059301A8FFF71EFD00B1FEE7F2
S3150800307011B05DF804FB08B5FFF7CCFFFFF748F978
S31508003080FFF7D0FF00F0B6F8FFF7ECF808BD08B573
S31508003090FFF7F1FFFFF780F8FFF7EEF8FFF7DEF826
S315080030A0FAE70000F0B589B03B4B9A6942F0010295
S315080030B09A619A6902F001020092009ADA6942F06E
S315080030C08052DA61DA6902F080520192019A9A69AD
S315080030D042F004029A619A6902F004020292029A84
S315080030E0DA6942F40032DA61DB6903F400330393E8
S315080030F0039B0320FFF730F9002211466FF00B00FF
S31508003100FFF73CF9002211466FF00A00FFF736F97F
S31508003110002211466FF00900FFF730F90022114628
S315080031206FF00400FFF72AF9002211466FF003003A
S31508003130FFF724F9002211466FF00100FFF71EF988
S31508003140002211464FF0FF30FFF718F920270497A1
S315080031500123059300250695022607960F4C04A918
S315080031602046FFF769F92A4639462046FFF75AFAF4
S315080031700423049305960323079304A92046FFF71F
S315080031805BF9082304930595069504A92046FFF7DD
S3150800319053F909B0F0BD00BF001002400008014015
S315080031A0DFF834D0002103E00C4B5B584350043160
S315080031B00B480C4B42189A42F6D30B4A02E00023FE
S315080031C042F8043B094B9A42F9D3FFF7FDFE00F09B
S315080031D031F8FFF75CFF704700500020C83200083E
S315080031E0000000200C0000200C000020BC0000207D
S315080031F0FEE7000008B5FFF713FD084BA3FB0030F8
S315080032008009FFF7EDF80420FFF700F900221146C0
S315080032104FF0FF30FFF7B2F808BD00BFD34D62107C
S3150800322008B5FFF793F808BD08B5FFF783F8FFF769
S31508003230FEF808BD70B500250C4E0D4CA41BA41055
S31508003240A54209D100F01AF800250A4E0A4CA41B1B
S31508003250A410A54205D170BD56F82530984701350A
S31508003260EEE756F8253098470135F2E7C0320008F0
S31508003270C0320008C0320008C4320008F8B500BFE2
S31508003280F8BC08BC9E467047F8B500BFF8BC08BC39
S309080032909E46704791
S3150800329402030405060708090A0B0C0D0E0F101085
S315080032A401020000000000000000000001020304FF
S311080032B4060708090000000001020304D8
S309080032C0352100089E
S309080032C411210008BE
S311080032C8010000001000000000A24A04EB
S705080031A120
